:1000000060284D0041005300090063001900000002
:10001000CA0015002F000100030000000000F200DC
:100020002F00C700BA00FF0043009400BD0003008A
:10003000410017008B00E4001600E600DC00B00071
:10004000C600FF003500B3000D0031006C005B00FE
:10005000BD00CF0048007B009E005300EC0028004C
:1000600043002900430041004E0041004C002B009A
:1000700031003900390034002F00390035002F00DD
:100080003900360020004E0075006D00340030004D
:1000900000003B00F7001100000001004000960046
:1000A0005400300004000E006C00B600D60084003E
:1000B0000000040000000000000016002100000005
:1000C0008A01CB20F0306500F0308500CA017F3016
:1000D0006200A301A401CB0149236830D02083161C
:1000E0009900990898168312031D98170030D020A4
:1000F000A3003030D020A4002C21031C82284B17F1
:1001000023112312CB120F30A31C0F3A231F85009B
:100110001730DB008530DC000030A1004930A20040
:100120000E30AF0002218A150A120028AF08031909
:100130000034AF039900C8003230CC2086137F30E2
:100140006600C9010830C600CB20C80C480C8039B5
:10015000C90606068606C60BA428CB204908060653
:100160008606CB20FF3066003E30CC28861BB628A2
:100170002D30CC200930C6000310861B0314C80C98
:10018000CB2000000000C60BBC28C80D1D30CC20C1
:100190004808990008001A30C700C70BCD28003462
:1001A00003178D0083168C130C1483120C08031391
:1001B00008000D1203178C000313220803178D008B
:1001C00083168C130C1555308D00AA308D008C14BD
:1001D000831203130D1EEA28831603170C118312D2
:1001E00003130800A5002F020318F928A507031917
:1001F00008002208B023A20A0319A10A9620A50B21
:10020000F9280800A500E5239620A20A0319A10AEF
:10021000A50B03290800A5002F0203181229A50722
:100220000319080000089620840AA50B122908006B
:10023000A5002F0203181F29A5070319080022088B
:10024000D0209620A20AA50B1F290800AF08031989
:100250000800FF30962026294321A0302F29A00036
:10026000CF3066000830C700A00D5621C70B3429D7
:100270005C29DF3066000830C7005E21A00DC70B87
:100280003D29031454290616CF3066008616000057
:10029000061252290612CF306600000086160000B2
:1002A0000616000086120800CF306600031C0612F6
:1002B0000318061686165129DF30660086160000E0
:1002C0000314061E0310522966216729C2006A2101
:1002D0006A216A21420884000008A00022088400E4
:1002E0000008A7002008800042088400270880003A
:1002F000A20AC20A0800C2000830C30042088400F3
:100300000008A0002208840020088000C20AA20A77
:10031000C30B7E29420808000030B800B900BA00BB
:10032000BB00BC00BD00BE00BF00B000B100B20009
:10033000B300B400B500B600B7000800003095293E
:100340008000840AA50BA02908005608031908009C
:1003500052220C30A500FF30B623A20A0319A10ACD
:10036000A50BAB290800C3001030A500AD01402249
:10037000013E0318A10AB023430603190034AD0A55
:10038000A50BB72902344022183E0318A10A5507CD
:10039000A2000318A10AB023D60008002E080F39C6
:1003A000103ED500C32152222208013EC20008009F
:1003B0000030A1000D30B02B0030A600D821DA00AB
:1003C000D601D60A52220B30A2070318A10A22082E
:1003D000B023A61BF229FF3A031908008039031D38
:1003E0000800F529260603190800D60A0C30A207D2
:1003F0000318A10ADA0BE7290800DC214022183E85
:100400000318A10A5507A2000318A10A5608B6232B
:1004100058180E2AD818252A5819372ACE214B1CCD
:10042000142A10302E07D1215708B6230A30A2070C
:100430000318A10A0030B623A20A0319A10A2D0845
:100440000F394B18C0388038B62B4E220830A2071F
:100450000318A10A0330A5000030B623A20A03192D
:10046000A10AA50B2C2A2D080F399038B62B522241
:100470000B30A2070318A10A2D080F39E038B62B5C
:100480000030A1002D080F39A700A70A40304B2AE1
:100490004B3E0318A10AA70B482A08000130D500DB
:1004A000C321522AA1015608A2000310A20DA10DDA
:1004B000A20DA10D210DA107220D0318A10AA2076B
:1004C0000318A10AF430A2070318A10A0430A107F7
:1004D000080030083107320733073407350736077D
:1004E00037075707FF3AD90008004208B0238000B9
:1004F000840A0730C300B3238000840AC30B7B2A1D
:1005000008004022163E0318A10AA20002302F2440
:10051000A319080002301B2C5124D7000F39AE005C
:100520002E245425692258142E084B18103EAE0074
:10053000103E8A150A124E278A110A12003A031D2C
:10054000FD21CE214B1CA72A10302E07D1214208B5
:10055000A200A31908001A245908B00001301B2476
:10056000492BB620AB00B620AC00B620AD00B620BB
:10057000AE00B620AF000800AA012F08031908003A
:10058000A500B6204224A50BC12A080008302F027E
:10059000A500AA00AA035124823A031D0134F122C6
:1005A000AA01E62229233A25A508031DD12ACA1447
:1005B000303084000830A50051240006031D0234A9
:1005C000840AA50BDC2A2923CA10003430308400A9
:1005D00051248006A50303190800840A841DE82A13
:1005E00008009E212D08E039A600203A0319012BAE
:1005F0002608403A0319112B2608603A03191E2BCE
:1006000008000030A1000230B023B000B323B100D5
:10061000B323B200B323B300B323B400B323B500B4
:1006200008004022123E0318A10AB023B000B323F1
:10063000B100B323B200B323B30008004022123E3E
:100640000318A10AB023B000B323B100B323B20052
:1006500008001F302D054006031D332B0F302E05DB
:1006600041060319442BCE21B030840075222D1E83
:100670003D2B10302E07103ED12175221F302D0545
:10068000C0000F302E05C100A030A200B0307B2189
:100690007B29FF30C000C1000800AE1F0800AA007F
:1006A00029232A0A2F02031C0800F839A500A508EF
:1006B000031908002E2454250830AA02A502382464
:1006C000572B2E08A2002D08A100A11F6A2B031092
:1006D000A20DA10D213A080061230319712B2F08E7
:1006E000F2282F081829BC22AA0161230319802BA4
:1006F0005124B623A20A0319A10AAF0B782B0800D4
:100700005124D920A20AAF0B802B08002D08A1008C
:100710002E08A200E52303170E08031396200317E3
:100720000C0803139620A20A0319A10AAF08031D9F
:100730008A2B0800BC222D08A1002E08A200AA01C5
:10074000AF0C512403178E000313512403178C00A0
:1007500003130024A20A0319A10AAF0BA12B08005E
:10076000231DDD2BB92B231DEC2BC32B231DF92BB4
:10077000CC2BA2004321A0302F210318BA2B210833
:100780002F2122082F214321A1302F210318C32B11
:1007900039214A212008080003178C000313432144
:1007A000A0302F210318CF2B21082F2122082F2121
:1007B00003170C0803132F214A2903178D00031375
:1007C0001030210703178F00EC2B220803178D0030
:1007D0000313210803178F00031783168C170C14BB
:1007E0000000000083120C088D0A03198F0A0313FE
:1007F000080003178C008E01031310302107012C11
:10080000210803178F000313220803178D00831696
:100810008C170C1555308D00AA308D008C14831266
:1008200003130D1E112C0D12831603170C118312C6
:10083000031308000830C900303084002208B023B8
:1008400000060319272C0008B623CC16CA15840A03
:10085000A20A0319A10AC90B1E2C08000830C900FE
:100860003030840051248000840AC90B322C0800E7
:100870000830C9003030840000084224840AC90BC3
:100880003C2C0800FF000408FE0090302A0784007A
:1008900083177F0880008313AA0A7E0884007F08DC
:1008A00008000408FE0090302A078400831700081F
:1008B000FF008313AA0A7E0884007F080800A801AD
:1008C000123084004E3C8313123E03190800831734
:1008D00000082606031D762C840A00082706031D3F
:1008E000772C840A00088313A8000800840A840A6D
:1008F000840A0408622C5F2428080319842C290820
:10090000831780008313080003171108033E91002A
:10091000900A10081A3C031D902C91019001842C20
:1009200011080F3E84000313260883178000840AF1
:1009300027088000840A29088000840A831308009D
:1009400003179001910103138317123084004E3076
:10095000A8008001840AA80BA92C8313080000308A
:10096000A1000A30B023A600B323A700B323A80038
:10097000CB1D241C08003430D020A6053530D020F3
:10098000A7050800AF242708AD192608C2002D08C6
:100990000739682603104205031D031408000130BF
:1009A000D500C321A521D50A5508303A031DD12C05
:1009B0004022A2004B30A500FF30B623A20A031943
:1009C000A10AA50BDC2C042D4022A2000030B62386
:1009D000A20A0319A10A3108B62310302207A20087
:1009E0000319A10A9E210730A5001A24A50BF52C96
:1009F00002301B24AF242D0807396826AD19022DBB
:100A0000A7040800A6040800AF242D0807396826AB
:100A1000FF3AAD190D2DA7050800A60508005222C2
:100A2000D230962000309620560896200C30F220C6
:100A3000003096200030962003309620CF0A4F08D1
:100A4000A60008005222D230962000309620560888
:100A500096202208B02396200830A500FF3096206B
:100A6000A50B2E2D2208093EA2000318A10A03306F
:100A7000F220182DA601A801BB25A80ABB25A80AAB
:100A8000BB25A80ABB250330A8027925A80A8D2515
:100A900026080F3A031908003030A20034306621CE
:100AA000A60A281AA8013C2DA801A601BB25A80A60
:100AB000280803390319A60A281F562D0F30A6004F
:100AC0000C30A80079258D25BB25A803BB25A803DC
:100AD000BB25A803BB25A608031908003030A200D7
:100AE00034306621A603FC30A8070C30A81BA800F0
:100AF000622DC7253406CD25C200A80AC7253506B4
:100B0000CD25C300A80AC7253606CD25C400A80AEE
:100B1000C7253706CD25C5000800C206450E440787
:100B2000D225C400C506440E4307D225C300C4061F
:100B3000430E4207D225C200C306420E4507CD250B
:100B4000C500C206450E4407CD25C400C506440EA7
:100B50004307CD25C300C4064208C3064308D22577
:100B6000B0064508D225B1064208D225B20644088F
:100B7000D225B3060800280AC825A7002803C825DF
:100B8000A706C72527082606CD25800608002808C1
:100B90000F39A03E8400000808008A150A16F825BF
:100BA0008A0108008A150A16FC258A010800231EFE
:100BB0000800231D08007C30D020A900DE007D3015
:100BC000D020A800DD007030D020A7007130D020E8
:100BD000A6000530AC1C2F07DD070318DE0A270826
:100BE0005E02031DF52D26085D020318432E043016
:100BF000A5002B3084007230A7002708D020A60063
:100C00000008A605A70A2708D0202606031D08000D
:100C1000840AA70AA50BFD2D2708D020000203197E
:100C2000132E03180800A70A2708D0200002031C6F
:100C300008007F30D02028070318A90AA2007E30C0
:100C4000D0202907A1004A152B30840000083D263A
:100C5000840A8419262EAC18342EAA012F08A50068
:100C600051243D26A50B302E7C30A2005E08D920F1
:100C70007D30A2005D08D9200800B623A20A031D1A
:100C80000800A10A0800CA150800E0302905803ACA
:100C9000031D0034A601A701290C07396826291C69
:100CA000A6002918A700FF30A6062308291A240841
:100CB00026052704291A622EA3000030A20023086B
:100CC000D9201034A4003030A2002408D9201034D8
:100CD0006B268A010800FF00F839031D0034073035
:100CE0008A007F08F83E82000030A1000530A20093
:100CF000443002218A150A12962F0030A1000030DC
:100D0000A2000830F2208A150A12962F4022A20073
:100D10001930F2208A150A12962F0301962003013A
:100D20009620AF242608962027089620280896208B
:100D3000510896208A150A12962FFF3FFF3FFF3F6A
:100D4000FF3FFF3FFF3FFF3FFF3FFF3FFF3FFF3FB3
:100D5000FF3FFF3FFF3FFF3FFF3FFF3FFF3FFF3FA3
:100D6000FF3FFF3FFF3FFF3FFF3FFF3FFF3FFF3F93
:100D7000FF3FFF3FFF3FFF3FFF3FFF3FFF3FFF3F83
:100FF0000134023404340834103420344034803452
:10100000AC01D101DA018A110A12A0248A150A1250
:101010009030C8270030C827A101CC01CB18CA14D2
:101020004A08A31C0F3A231F85002C08D3003C3A22
:1010300003191C28CB18D301CB108A110A12B12234
:101040008A150A12C1302B06031D7F282F085F3C2A
:10105000031C902FAF08031D3028AC18932F3228A3
:101060002C08C827CB1D44282C08203A0319982B9C
:10107000023A03199E2B063A0319A42B023A0319CC
:10108000AA2B2A3A0319832B2C08403A031D562811
:101090002D08031D56282E08803A031D56282F08B8
:1010A000031D5628CB154030C827962FAC185D2855
:1010B0008A110A12BC228A150A128A110A12D7252D
:1010C0008A150A121A30C30043080E3ED4272C0694
:1010D00003196E28C30B6428CC1572284308033CFF
:1010E000031879288A110A12C2248A150A12031CCD
:1010F0009C2FCC1D82284A15AC18EC27932F4A153B
:101100006E300928D001D2014A1108308A00430804
:10111000893E8200A428A728642BAD28AA28A12AEA
:101120007129E728BD2ACE2AF32AB028102B222BBA
:101130002F2B442B452B822B562B5D2B5E2B5E2BAE
:101140005E2B5E2B5F2B822B8A110A12742E8A1162
:101150000A127D2E8A110A12862E8A110A128D2EEB
:101160003030A900A801AE014927003A031DC92863
:10117000290884002E088A110A1252228A150A129E
:1011800022088A110A12B0238A150A128000A90ABD
:10119000A80AAE0A2E1EB4284027A2008A110A12FD
:1011A000B0239620B32396200C3096206C309620E6
:1011B000B32396208A150A123030840028080319B8
:1011C000E6288A110A120B218A150A12962F2E0878
:1011D0000319F128013A03193029033A0319442964
:1011E000C02F2F08103A031D902F5721003A0319E2
:1011F0000A29A41D632F2608270428042904031D97
:10120000A62F5308323A031DA62F4D08033A031D9B
:10121000A62F2029A808031D1829A9080319182991
:101220008A110A1245268A150A12003A031D632FF5
:1012300028082606031D222929082706031D22291E
:101240005927C42F0E30AA002E30A2008A110A128C
:101250005124D920A20A5124D9208A150A12962F86
:101260002F08093A031D902F5721003A031D632FC1
:101270000830AA00DA27A8000030A1000830043E98
:10128000A2002808E027962F2F08093A031D902F67
:101290005721003A031D632F0830AA00DA27D10036
:1012A0005118D101511AD101D11AD101962F06300E
:1012B000AA00DA27A600DA27A70028040319CA0122
:1012C0000E30AA00DA27A800DA27A9002E30D4278A
:1012D0002606031D10342F30D4272706031D103493
:1012E0000034AE08031DC02F3430530603197C2987
:1012F00032305306031DAC2F4D08003A0319D7298D
:10130000013A03198D29023A0319E929073A031909
:10131000802A023A03199D29AE2F2D0803199A2914
:101320000030A1005730A20009308A110A120221B0
:101330008A150A120430CE27962FCF0803199A294E
:101340008A110A12D8218A150A12DA004F08D6002B
:101350005A02031C9A298A110A1252228A150A1269
:101360000B302207A2000318A10AE627A7000F39B5
:101370002D060319C129CF0ADA0BA6292608CF00AA
:101380009A29CB19CB292708F039803A0319D1299A
:10139000403A0319D1298A110A120F258A150A1217
:1013A0009C298A110A1222258A150A129C29AD0845
:1013B00003199A2901304E27003A031D9A298A11F0
:1013C0000A12833096204E220830F2208A150A1223
:1013D0009A29AD0803199A29CE08031DF229CF08CE
:1013E00003193B2A231CF6294B1E9A29A31B112AF9
:1013F0004E08B200A6004F08B100A7002D080F3913
:10140000B038BB007E25003A031D9A298A110A12C2
:1014100052228A150A125C226E2275220330CE27D0
:101420009C294E08A6004F08A7008A110A125F24C3
:101430008A150A12A808031D1E2AA8038A110A1277
:10144000B1309620030196204E0896204F08962032
:10145000280896200130962003019620030196204B
:101460005B0896205C0896200301962003019620D5
:101470008A150A129A29DA0803199A290C302F02C0
:101480000319592A031C592A2D080F39B038A60010
:101490008A110A12E1218A150A12DA0803199A2917
:1014A0008A110A1252228A150A125C226E227522B1
:1014B0003B2A0330CE279C29303084002208E627BF
:1014C0008000840A0A30C3008A110A12B3238A15E5
:1014D0000A128000840AC30B642A08003108C30082
:1014E0003208B1004308B20008008A110A12B13074
:1014F0009620303084000B300B218A150A12080028
:10150000AD08031D9A294F08003A03198E2A013AA3
:1015100003199D2A033A03199F2A9A2904304E275A
:10152000003A031D9A298A110A125222B2309620DB
:101530000B30F2208A150A129A2902308F2A0330C2
:101540008F2AFF30CD002F08033A031D902F033060
:10155000A5004D308400AA01DA278000840AA50B7B
:10156000AC2A5308303A03194B168A110A12D821B3
:101570008A150A12DA00D601962F4A103C3053061B
:10158000031DAC2FAA011030A5008A110A125124A4
:1015900096208A150A12A50BC52A962F4B124A14BB
:1015A0004927003A031DB22F8A110A122923083055
:1015B0004D23C6228A150A12003A0319E12A023085
:1015C000E72AB023003A0319632F4C18632FA900B0
:1015D0008A110A12FF309521AA01382438248A156D
:1015E0000A122908632FAE19AA2F4927003A031DB2
:1015F000B22F8A110A12292303014D23C6228A150C
:101600000A12003A031D982F4A14B023003A031D12
:10161000632F4C1AAE2F4C1BB02FCC1BC42F962F10
:101620004927003A031DB22F2E1AC02F8A110A1221
:1016300029239E213A253030840008300B218A1559
:101640000A12962F04305306031DAC2F303084004D
:1016500008308A110A120B218A150A12962F2F08B8
:10166000083A031D902F4927003A031DB22F2E0878
:101670000F390F3A031DB82F8A110A1229232E247D
:101680003A258A150A12962FAC2F4A144927003A98
:101690000319B22F8A110A12292303014D23C622EE
:1016A0008A150A12003A031D982F962FDA27A700F1
:1016B000271A5116A71AD116962F962FA82F2F0842
:1016C000083A031D902F962F2F08033A031D902FE1
:1016D000DA27DA27A600DA27A70003302602031C40
:1016E000752B031D752BE8302702031CC62F3230E3
:1016F0002602031C7F2B031D7F2BC93027020318F2
:10170000C62F962FAC2F8A110A12BC228A150A12F4
:10171000AA012F08083A031D902F8A110A122E24BD
:101720000030A1000030A2001A248A150A12962F58
:101730008A110A126C238A150A12962F8A110A122C
:1017400073238A150A12962F8A110A1286238A1584
:101750000A12962F8A110A129A238A150A12962FB4
:10176000AA01CB13D8012A082F0203190034DA2763
:10177000A600D00A2C1FFD2B2608013A0319262C9F
:10178000033A0319392C013A0319482C133A031967
:101790005D2C013A0319792C063A03199B2C363A31
:1017A0000319AD2C033A0319B52C103A03194A2D2D
:1017B000723A0319A42D013A0319B72DD13A03192E
:1017C000CC2D013A0319D52D213A0319D72D603AB2
:1017D0000319F92D203A03190B2E703A0319582ECC
:1017E000A33A0319D42C073A0319022D013A03191D
:1017F000242D033A0319382D162C2608043A031910
:101800007B2E173A03197C2E0A3A0319A12E3E3A71
:101810000319A42E163A0319CE2EE03A0319032F0A
:10182000203A0319192F733A03191A2F260E0F396C
:101830001B24AA07B22B0D3A03191034033A0319DB
:101840001834013A031920340F3A08003527B01F25
:1018500008344027023E0318A10AA200FF30B0005E
:1018600001308A110A121B248A150A12CC1E59272C
:10187000B22B4027023E0318A10AA200B00101309A
:101880008A110A121B248A150A12CC1E5927B22B60
:101890002E30D427A6002F30D427A7002604031902
:1018A000B22B8A110A122E30A2000030D920A20ACF
:1018B0000030D9208A150A12B22BDA270F39AE0070
:1018C0006F248A110A12A5218A150A122E08103EC9
:1018D0006F248A110A12A5218A150A12B22B8A11C5
:1018E0000A12103ED500C3210030B6238A150A1211
:1018F00008000130F2273008003A0319862C013A1B
:1019000003198A2C033A0319882CB22B04308B2C30
:1019100003308B2C02304E27003A031DB22B8A1164
:101920000A12A521C3210030B6238A150A12B22B50
:10193000CC1E5927B22B8A110A124022183E0318D6
:10194000A10AA2000318A10A01302F2401301B2490
:101950008A150A12CC1E5927B22B8A110A1281222B
:101960008A150A12CC1E5927B22B2419192C8A1158
:101970000A124022163E0318A10AB023A800B3237E
:10198000A9005124A6005124A7008A150A1228088C
:101990002602031CCF2C031DCF2C29082702031974
:1019A000D32C03183134B22BAD08031D053402309B
:1019B000F22731088A110A12B3218A150A12003A55
:1019C00003191834FF308A110A12B3218A150A123A
:1019D000003A031D06348A110A12DC218A150A1204
:1019E0005608E73A031919348A110A12E4248A15B1
:1019F0000A120A30A2002608E027A20A2708E027D8
:101A0000CB17B22BAD08031D05340230F227B00806
:101A1000031D043431088A110A12B3218A150A12EF
:101A2000003A031D04348A110A12C2248A150A12CC
:101A3000031C04344027023E0318A10AE627FF3A9C
:101A400003190734CB17B22BAD08031D0534023040
:101A5000F2278A110A12B3218A150A12003A031DCD
:101A600004348A110A12CF248A150A12F92CB22BD7
:101A7000CB1B3D2DAD08031D05340230F227402756
:101A8000A20002308A110A121B248A150A12CC1EE7
:101A90005927B22B35273019502D4C160330192CED
:101AA0008A110A128C215124B2005124B100512410
:101AB000B400FF30B300B700B8002D080F39B038BC
:101AC000BB008A150A12B208031D692DB10803195B
:101AD000B22B7E25003A031900348A110A12DC2148
:101AE0008A150A125608E73A031903348A110A12B2
:101AF00052220C301B248A150A12B22B2D080F39E2
:101B0000B0388A110A12DD218A150A12DA0803197F
:101B100002348A110A1252228A150A12A20A0319E1
:101B2000A10A2208E6273106031D9E2D8A110A12FA
:101B3000B3238A150A123206031900348A110A12D5
:101B4000E1218A150A12862D0430F2272D080F395B
:101B5000B0388A110A12DD218A150A12DA0803192F
:101B6000B22B8A110A12A5218A150A12A62D8A11F2
:101B70000A124022123E0318A10AA2000318A10A69
:101B800004302F2404301B248A150A12CC1ACA2DC3
:101B90005927B22B4C17B22B4B108A110A128C22E8
:101BA0008A150A12CC1E5927B22B4B14CD2D0B309F
:101BB000F227AD08031DE72D58153008003A031928
:101BC000E82D013A0319EC2D033A0319EA2DB22B43
:101BD0000430ED2D0330ED2D02304E278A110A120C
:101BE000003A031DFD2152220B301B248A150A12D4
:101BF000B22B8A110A124022023E0318A10AA20047
:101C00000318A10A2E241A242E241A248A150A1233
:101C1000CC1E5927B22B2A08203EA8008A110A128E
:101C200040228A150A12153E0318A10AE627A600CB
:101C300047260318442EA31A212EA6080319442E62
:101C400009342608A900A90A03192B2E29084726BA
:101C50000318382E232E26080319442EA900A903A1
:101C6000290847260318382E29080319202E2F2E5D
:101C70008A110A1240228A150A12153E0318A10A77
:101C8000A2002908E027CA152808AA00B22BA7003D
:101C90000739A500A70CA70C270C1F392802AA009A
:101CA000AA03DA27A700A50AA70CA50B542E080043
:101CB000241A792E3527301A602E4C160830192C2C
:101CC0000830A5008A110A124E228A150A125608F7
:101CD000003A031D722ED8148A110A12FD214E22D9
:101CE0008A150A128A110A122E241A248A150A1237
:101CF000CC1E5927B22B262FDA27A600C039031D88
:101D0000B22BA4189F2E8A110A124E228A150A128B
:101D10002608A500F839A6000310A60CA60C260C70
:101D20002202073EA2000318A10AE627A600250802
:101D30000739A500A50AA60CA50B9B2E0318262F74
:101D4000B22BDA274C14262F8A110A124022163E93
:101D50000318A10AB023A800B323A9005124A600A8
:101D60005124A7008A150A1228082602031CBC2E3B
:101D7000031DBC2E290827020319C02E0318313475
:101D80002708DB002808DC00B22B8A110A125F2426
:101D90008A150A12280803191A34E12EDA27A60038
:101DA000B200DA27A700B100DA27A900A31FE72EA7
:101DB000231CE12E1B27031DE12E5308303A031D7F
:101DC000C52E8A110A127B248A150A12262F7E2517
:101DD000003A031DB22B8A110A1252228A150A12E6
:101DE0005C222908B300340A031DF82E0130B40028
:101DF0005B08B7005C08B8000B308A110A121B247C
:101E00008A150A12262F32348A110A1229232E2407
:101E100054252A08A900AA0138242908AA002E243A
:101E200054250830AA0038248A150A124C1C0034A4
:101E30002734162C60342A08DE00DA27DD005E081D
:101E4000AA005D082C3A0319013400342A082F0235
:101E500003196F34DA27A600D00AD13A0319042FE8
:101E6000260E0F391B24AA07262F4027A2008A110D
:101E70000A12B023B000B323B1008A150A12080079
:101E80008A110A1240228A150A12483E0318A10A32
:101E900008002E080F392D1A103E103ED5008A1169
:101EA0000A12C3218A150A125608003A031902348D
:101EB000003450038A110A1268268A150A12D204C5
:101EC000CC12CC170800CA10A900AC18EC272908BE
:101ED0002F3C03187A2F290E0F39063A0319802F49
:101EE000013A03198C2F073A903EC827CB142908D2
:101EF0000F390B289030C8272908031DCB140B2855
:101F0000CA149630C82729080F390F3A03198A2FA7
:101F10000F3A0B2850080B289730C82752080B2877
:101F20006730CB1409286D30CB1409280301632FC7
:101F30000230632F0330632F0430632F0530632F8B
:101F40000730632F0830632F0930632F1030632F61
:101F50001130632F1330632F1430632F1530632F2C
:101F60001930632F2D1AB62F1D30632F1F30632FAA
:101F70002130632F3130632F3230632F3430632FA1
:101F80004230632F6F30632F7030632F8130632FA7
:101F90008A110A129A208A150A1208008A110A1256
:101FA00096208A150A1208008A110A12D0208A1572
:101FB0000A1208008A110A1251248A150A1208000E
:101FC0008A110A12B6238A150A1208008A110A1207
:101FD000B0238A150A1208008A110A1226218A15CE
:101FE0000A1208008A110A122F248A150A12080000
:101FF0008A110A1229238A150A120800FF3FFF3F9F
:102000000000250000000000000007005B00CD007C
:1020100000000000000001000000BF00FF3FFF3F84
:10202000FF3FFF3FFF3FFF3FFF3FFF3FFF3FFF3FC0
:10203000FF3FFF3FFF3FFF3FFF3FFF3FFF3FFF3FB0
:10204000FF3FFF3FFF3FFF3FFF3FFF3FFF3FFF3FA0
:10205000FF3FFF3FFF3FFF3FFF3FFF3FFF3FFF3F90
:10206000FF3FFF3FFF3FFF3FFF3FFF3FFF3FFF3F80
:10207000FF3FFF3FFF3FFF3FFF3FFF3FFF3FFF3F70
:1020800000000000530045004300410020002000F4
:102090002000200020002000200020002000200040
:1020A00020002000000000000000000000000000F0
:1020B000000000000100020003000000000000001A
:1020C0000000000000000000000000000000000010
:1020D00004000000000000000000000000000000FC
:1020E00000000000000000000000000000000000F0
:1020F00005000000000000000000000000000000DB
:1021000000000000000000000000000000000000CF
:10211000FF00FF000000FF3FFF3FFF3FFF3FFF3F8B
:10212000FF3FFF3FFF3FFF3FFF3FFF3FFF3FFF3FBF
:10213000FF3FFF3FFF3FFF3FFF3FFF3FFF3FFF3FAF
:10214000FF3FFF3FFF3FFF3FFF3FFF3FFF3FFF3F9F
:10215000FF3FFF3FFF3FFF3FFF3FFF3FFF3FFF3F8F
:102A000001000000000000000000000000000000C5
:102A1000020089009B00E000020028000500190068
:102A20009800000000000000000000000000E0002E
:102A300000000400050000001B0000000C00030063
:102A40003C0082002200E000F000000000000000D6
:102A5000000000000000000000000F0000008000E7
:102A60005000000000000000000000000000000016
:102A700000000F000000C000FF3FFF3FFF3FFF3F8F
:102A8000FF3FFF3FFF3FFF3FFF3FFF3FFF3FFF3F56
:102A9000FF3FFF3FFF3FFF3FFF3FFF3FFF3FFF3F46
:102AA000FF3FFF3FFF3FFF3FFF3FFF3FFF3FFF3F36
:102AB000FF3FFF3FFF3FFF3FFF3FFF3FFF3FFF3F26
:103BF0000A108A140A1582000A148A140A1582000F
:103C00002A34E1340B3413343E346E3432344834C5
:103C1000D334313408348C348F349534BD34D034BB
:103C2000E4346D345034813420343034BB34753452
:103C3000F534D4347C3487342C344E34E834F434C2
:103C4000BE3424349E344D3480343734D2345F341F
:103C5000DB3404347A343F341434723467342D3412
:103C6000CD341534A6344C342E343B340C3441342A
:103C70006234FA34EE3483341E34A23401340E3408
:103C80007F345934C934B934C4349D349B341B3423
:103C90009C34CA34AF343C3473341A346534B13490
:103CA0007634843439349834E93453349434BA341F
:103CB0001D342934CF34B4340D3405347D34D1343B
:103CC000D7340A34A0345C3491347134923488345B
:103CD000AB34933411348A34D6345A347734B5340F
:103CE000C3341934C134C7348E34F934EC34353428
:103CF0004B34CC34D9344A34183423349F345234BE
:103D0000DD34E334AD347B344734973460341034DD
:103D10004334EF340734A5344934C634B33455340E
:103D2000283451345D3464346634FC3444344234D1
:103D3000BC342634093474346F34F7346B344F3464
:103D40002F34F034EA34B834AE34F33463346A34A4
:103D50005634B2340234D8343434A4340034E63423
:103D60005834EB34A334823485344534E034893418
:103D70007E34FD34F2343A3436345734FF3406346A
:103D80006934543479349A34B6346C34DC348B343A
:103D9000A7341F349034033417341C34ED34D53435
:103DA000AA345E34FE34DA347834B034BF3412349A
:103DB000A834223421343D34C234C034B734A93459
:103DC000E7343334FB34F1347034E534173496344B
:103DD000F8348D344634A1348634E23440343834F7
:103DE000F634683425341634AC3461342734CB349B
:103DF0005B34C8342B340F349934DE34CE34C534BC
:103E0000BF3411346D34FA3426347F34F334C8347B
:103E10009E34DD343F3416349734BD340834803456
:103E200051344234933449345B3464349B34253404
:103E3000F5340F34243434344434B834EE342E346E
:103E4000DA348F343134CC34C0345E348A34613463
:103E5000A1346334C734B234583409344D34463451
:103E60008134823468344B34F634BC349D340334AA
:103E7000AC349134E8343D3494343734A034BB341A
:103E8000CE34EB349834D83438345634E9346B3487
:103E90002834FD348434C634CD345F346E34B634C3
:103EA0003234F7340E34F134F8345434C1345334EA
:103EB000F034A73495347B341934213423347D34E1
:103EC000E134A93475343E34D634ED348E346F3455
:103ED000DB34B7340734413405347734B4342D340B
:103EE0004534DF3429342234433489348334FC3478
:103EF000D534A4348834D134F43455344F34783440
:103F000062341E341D34B934E0342F340134133498
:103F10001534E63417346A348D340C3496347E34D8
:103F200086342734A6340D34B53473347134AA344E
:103F30003634D03406346634DC34B1342A345A345E
:103F40007234BE343A34C534403465341B340234E0
:103F500010349F343B34F9342B3418345C34D73468
:103F600012344734EF341A348734D234C2348B34A9
:103F700099349C34D3345734E43476346734CA34B7
:103F80003C34FB349034203414344834C934603425
:103F9000B03470344E34A234AD343534EA34C434E1
:103FA0007434CB343934DE34E734D434A334A53418
:103FB000043492348C34D9347C341C347A34A834AC
:103FC00052347934F2343334BA341F3430349A34BE
:103FD000003450344C34FF34E534CF345934C334D6
:103FE000E3340A348534B334AE34EC340B34FE3469
:103FF000E234AB344A34AF3469346C342C345D343D
:084000000F000F000F000F007C
:02400E00393F38
:1042000081006D006F0073006300410053003100B6
:1042100032003300200020002000170085000A0033
:104220000E007C00160012003400320030003A000C
:104230003C0040001A005A0002000400360038001A
:10424000420048004A004C005000540056005C00F8
:104250008A00FF00FF00FF00FF00FF0000000000D9
:10426000000000000000000000000300FF00FF004D
:10427000FF00FF00FF00FF00FF00FF00FF00FF0046
:10428000FF00FF00FF00FF00FF00FF00FF00FF0036
:10429000FF00FF00FF00FF00FF00FF00FF00FF0026
:1042A000FF00FF00FF00FF00FF00FF00FF00FF0016
:1042B000FF00FF00FF00FF00FF00FF00FF00FF0006
:1042C000FF00FF00FF00FF00FF00FF00FF00FF00F6
:1042D0000500FF00FF00FF00FF00FF00FF00FF00E0
:1042E00004000000FF000000FF000000FF000000CD
:1042F000FF000000FF000000000000000C000000B4
:10430000FF00FF00FF00FF00FF00FF00FF00FF00B5
:10431000FF00FF00FF00FF00FF00FF00FF00FF00A5
:10432000FF00FF00FF00FF00FF00FF00FF00FF0095
:10433000FF00FF00FF00FF00FF00FF00FF00FF0085
:10434000FF00FF00FF00FF00FF00FF00FF00FF0075
:10435000FF00FF00FF00FF00FF00FF00FF00FF0065
:10436000FF00FF00FF00FF00FF00FF00FF00FF0055
:10437000FF00FF00FF00FF00FF00FF00FF00FF0045
:10438000FF00FF00FF00FF00FF00FF00FF00FF0035
:10439000FF00FF00FF00FF00FF00FF00FF00FF0025
:1043A000FF00FF00FF00FF00FF00FF00FF00FF0015
:1043B000FF00FF00FF00FF00FF00FF00FF00FF0005
:1043C000FF00FF00FF00FF00FF00FF00FF00FF00F5
:1043D000FF00FF00FF00FF00FF00FF00FF00FF00E5
:1043E000FF00FF00FF00FF00FF00FF00FF00FF00D5
:1043F000FF00FF00FF00FF00FF00FF00FF00FF00C5
:00000001FF
